 management

 Timestamp is 6710e055 (Thu Oct 17 10:00:53 2024)

 Preferred load address is 10000000

 Start         Length     Name                   Class
 0001:00000000 000031d3H .text$mn                CODE
 0002:00000000 0000013cH .idata$5                DATA
 0002:0000013c 00000008H .00cfg                  DATA
 0002:00000144 00000004H .CRT$XCA                DATA
 0002:00000148 00000004H .CRT$XCZ                DATA
 0002:0000014c 00000004H .CRT$XIA                DATA
 0002:00000150 00000004H .CRT$XIZ                DATA
 0002:00000154 00000004H .CRT$XPA                DATA
 0002:00000158 00000004H .CRT$XPZ                DATA
 0002:0000015c 00000004H .CRT$XTA                DATA
 0002:00000160 00000010H .CRT$XTZ                DATA
 0002:00000164 00000000H .gfids$y                DATA
 0002:00000170 00000a10H .rdata                  DATA
 0002:00000b80 00000000H .rdata$CastGuardVftablesA DATA
 0002:00000b80 00000000H .rdata$CastGuardVftablesC DATA
 0002:00000b80 00000004H .rdata$sxdata           DATA
 0002:00000b84 0000006cH .rdata$voltmd           DATA
 0002:00000bf0 000002f4H .rdata$zzzdbg           DATA
 0002:00000ee4 00000004H .rtc$IAA                DATA
 0002:00000ee8 00000004H .rtc$IZZ                DATA
 0002:00000eec 00000004H .rtc$TAA                DATA
 0002:00000ef0 00000008H .rtc$TZZ                DATA
 0002:00000ef8 00000088H .xdata$x                DATA
 0002:00000f80 000019b8H .edata                  DATA
 0002:00002938 000000dcH .idata$2                DATA
 0002:00002a14 00000014H .idata$3                DATA
 0002:00002a28 0000013cH .idata$4                DATA
 0002:00002b64 000006c8H .idata$6                DATA
 0003:00000000 00000068H .data                   DATA
 0003:00000068 0000040cH .bss                    DATA
 0004:00000000 00000060H .rsrc$01                DATA
 0004:00000060 00000328H .rsrc$02                DATA

  Address         Publics by Value              Rva+Base       Lib:Object

 0000:00000000       ___AbsoluteZero            00000000     <absolute>
 0000:00000000       ___arm64x_extra_rfe_table  00000000     <absolute>
 0000:00000000       ___arm64x_extra_rfe_table_size 00000000     <absolute>
 0000:00000000       ___arm64x_native_entrypoint 00000000     <absolute>
 0000:00000000       ___arm64x_redirection_metadata 00000000     <absolute>
 0000:00000000       ___arm64x_redirection_metadata_count 00000000     <absolute>
 0000:00000000       ___dynamic_value_reloc_table 00000000     <absolute>
 0000:00000000       ___enclave_config          00000000     <absolute>
 0000:00000000       ___guard_check_icall_a64n_fptr 00000000     <absolute>
 0000:00000000       ___guard_eh_cont_count     00000000     <absolute>
 0000:00000000       ___guard_eh_cont_table     00000000     <absolute>
 0000:00000000       ___guard_fids_count        00000000     <absolute>
 0000:00000000       ___guard_fids_table        00000000     <absolute>
 0000:00000000       ___guard_iat_count         00000000     <absolute>
 0000:00000000       ___guard_iat_table         00000000     <absolute>
 0000:00000000       ___guard_longjmp_count     00000000     <absolute>
 0000:00000000       ___guard_longjmp_table     00000000     <absolute>
 0000:00000000       ___hybrid_auxiliary_delayload_iat 00000000     <absolute>
 0000:00000000       ___hybrid_auxiliary_delayload_iat_copy 00000000     <absolute>
 0000:00000000       ___hybrid_auxiliary_iat    00000000     <absolute>
 0000:00000000       ___hybrid_auxiliary_iat_copy 00000000     <absolute>
 0000:00000000       ___hybrid_code_map         00000000     <absolute>
 0000:00000000       ___hybrid_code_map_count   00000000     <absolute>
 0000:00000000       ___hybrid_image_info_bitfield 00000000     <absolute>
 0000:00000000       ___x64_code_ranges_to_entry_points 00000000     <absolute>
 0000:00000000       ___x64_code_ranges_to_entry_points_count 00000000     <absolute>
 0000:00000001       ___safe_se_handler_count   00000001     <absolute>
 0000:00000100       ___guard_flags             00000100     <absolute>
 0000:00000000       ___ImageBase               10000000     <linker-defined>
 0001:00000000       _Java_sun_management_ClassLoadingImpl_setVerboseClass@12 10001000 f   ClassLoadingImpl.obj
 0001:00000015       _Java_sun_management_DiagnosticCommandImpl_executeDiagnosticCommand@12 10001015 f   DiagnosticCommandImpl.obj
 0001:0000002b       _Java_sun_management_DiagnosticCommandImpl_getDiagnosticCommandInfo@12 1000102b f   DiagnosticCommandImpl.obj
 0001:000001e2       _Java_sun_management_DiagnosticCommandImpl_getDiagnosticCommands@8 100011e2 f   DiagnosticCommandImpl.obj
 0001:000001f4       _Java_sun_management_DiagnosticCommandImpl_setNotificationEnabled@12 100011f4 f   DiagnosticCommandImpl.obj
 0001:0000022b       _getDiagnosticCommandArgumentInfoArray 1000122b f   DiagnosticCommandImpl.obj
 0001:00000371       _Java_sun_management_FileSystemImpl_init0@8 10001371 f   FileSystemImpl.obj
 0001:00000374       _Java_sun_management_FileSystemImpl_isAccessUserOnly0@12 10001374 f   FileSystemImpl.obj
 0001:0000040e       _Java_sun_management_FileSystemImpl_isSecuritySupported0@12 1000140e f   FileSystemImpl.obj
 0001:000006ba       _Java_sun_management_Flag_getAllFlagNames@8 100016ba f   Flag.obj
 0001:000006c9       _Java_sun_management_Flag_getFlags@20 100016c9 f   Flag.obj
 0001:000008cb       _Java_sun_management_Flag_getInternalFlagCount@8 100018cb f   Flag.obj
 0001:000008de       _Java_sun_management_Flag_initialize@8 100018de f   Flag.obj
 0001:0000095a       _Java_sun_management_Flag_setBooleanValue@16 1000195a f   Flag.obj
 0001:00000980       _Java_sun_management_Flag_setDoubleValue@20 10001980 f   Flag.obj
 0001:000009a8       _Java_sun_management_Flag_setLongValue@20 100019a8 f   Flag.obj
 0001:000009c6       _Java_sun_management_Flag_setStringValue@16 100019c6 f   Flag.obj
 0001:00000a0e       _Java_sun_management_GarbageCollectorImpl_getCollectionCount@8 10001a0e f   GarbageCollectorImpl.obj
 0001:00000a23       _Java_sun_management_GarbageCollectorImpl_getCollectionTime@8 10001a23 f   GarbageCollectorImpl.obj
 0001:00000a38       _Java_sun_management_GarbageCollectorImpl_setNotificationEnabled@16 10001a38 f   GarbageCollectorImpl.obj
 0001:00000a74       _Java_sun_management_GcInfoBuilder_fillGcAttributeInfo@28 10001a74 f   GcInfoBuilder.obj
 0001:00000bfc       _Java_sun_management_GcInfoBuilder_getLastGcInfo0@32 10001bfc f   GcInfoBuilder.obj
 0001:00000e8b       _Java_sun_management_GcInfoBuilder_getNumGcExtAttributes@12 10001e8b f   GcInfoBuilder.obj
 0001:00000ebc       _Java_sun_management_HotSpotDiagnostic_dumpHeap0@16 10001ebc f   HotSpotDiagnostic.obj
 0001:00000ed3       _Java_sun_management_HotspotThread_getInternalThreadCount@8 10001ed3 f   HotspotThread.obj
 0001:00000ee6       _Java_sun_management_HotspotThread_getInternalThreadTimes0@16 10001ee6 f   HotspotThread.obj
 0001:00000efd       _Java_sun_management_MemoryImpl_getMemoryManagers0@8 10001efd f   MemoryImpl.obj
 0001:00000f0e       _Java_sun_management_MemoryImpl_getMemoryPools0@8 10001f0e f   MemoryImpl.obj
 0001:00000f1f       _Java_sun_management_MemoryImpl_getMemoryUsage0@12 10001f1f f   MemoryImpl.obj
 0001:00000f32       _Java_sun_management_MemoryImpl_setVerboseGC@12 10001f32 f   MemoryImpl.obj
 0001:00000f47       _Java_sun_management_MemoryManagerImpl_getMemoryPools0@8 10001f47 f   MemoryManagerImpl.obj
 0001:00000f72       _Java_sun_management_MemoryPoolImpl_getCollectionUsage0@8 10001f72 f   MemoryPoolImpl.obj
 0001:00000f7a       _Java_sun_management_MemoryPoolImpl_getMemoryManagers0@8 10001f7a f   MemoryPoolImpl.obj
 0001:00000fa5       _Java_sun_management_MemoryPoolImpl_getPeakUsage0@8 10001fa5 f   MemoryPoolImpl.obj
 0001:00000fd0       _Java_sun_management_MemoryPoolImpl_getUsage0@8 10001fd0 f   MemoryPoolImpl.obj
 0001:00000ffb       _Java_sun_management_MemoryPoolImpl_resetPeakUsage0@8 10001ffb f   MemoryPoolImpl.obj
 0001:0000101a       _Java_sun_management_MemoryPoolImpl_setCollectionThreshold0@24 1000201a f   MemoryPoolImpl.obj
 0001:0000107f       _Java_sun_management_MemoryPoolImpl_setPoolCollectionSensor@12 1000207f f   MemoryPoolImpl.obj
 0001:0000109b       _Java_sun_management_MemoryPoolImpl_setPoolUsageSensor@12 1000209b f   MemoryPoolImpl.obj
 0001:000010b7       _Java_sun_management_MemoryPoolImpl_setUsageThreshold0@24 100020b7 f   MemoryPoolImpl.obj
 0001:0000113c       _Java_sun_management_OperatingSystemImpl_getCommittedVirtualMemorySize0@8 1000213c f   OperatingSystemImpl.obj
 0001:0000117b       _Java_sun_management_OperatingSystemImpl_getFreePhysicalMemorySize0@8 1000217b f   OperatingSystemImpl.obj
 0001:000011b0       _Java_sun_management_OperatingSystemImpl_getFreeSwapSpaceSize0@8 100021b0 f   OperatingSystemImpl.obj
 0001:000011e5       _Java_sun_management_OperatingSystemImpl_getProcessCpuLoad0@8 100021e5 f   OperatingSystemImpl.obj
 0001:00001252       _Java_sun_management_OperatingSystemImpl_getProcessCpuTime0@8 10002252 f   OperatingSystemImpl.obj
 0001:0000129f       _Java_sun_management_OperatingSystemImpl_getSystemCpuLoad0@8 1000229f f   OperatingSystemImpl.obj
 0001:000012f9       _Java_sun_management_OperatingSystemImpl_getTotalPhysicalMemorySize0@8 100022f9 f   OperatingSystemImpl.obj
 0001:0000132e       _Java_sun_management_OperatingSystemImpl_getTotalSwapSpaceSize0@8 1000232e f   OperatingSystemImpl.obj
 0001:00001363       _Java_sun_management_OperatingSystemImpl_initialize0@8 10002363 f   OperatingSystemImpl.obj
 0001:0000138a       ___local_stdio_printf_options 1000238a f i OperatingSystemImpl.obj
 0001:00001390       __snprintf                 10002390 f i OperatingSystemImpl.obj
 0001:000013aa       __vsnprintf                100023aa f i OperatingSystemImpl.obj
 0001:000013c5       __vsnprintf_l              100023c5 f i OperatingSystemImpl.obj
 0001:00001e64       _Java_sun_management_ThreadImpl_dumpThreads0@24 10002e64 f   ThreadImpl.obj
 0001:00001e85       _Java_sun_management_ThreadImpl_findDeadlockedThreads0@8 10002e85 f   ThreadImpl.obj
 0001:00001e96       _Java_sun_management_ThreadImpl_findMonitorDeadlockedThreads0@8 10002e96 f   ThreadImpl.obj
 0001:00001ea5       _Java_sun_management_ThreadImpl_getThreadAllocatedMemory0@16 10002ea5 f   ThreadImpl.obj
 0001:00001ebc       _Java_sun_management_ThreadImpl_getThreadAllocatedMemory1@16 10002ebc f   ThreadImpl.obj
 0001:00001ed3       _Java_sun_management_ThreadImpl_getThreadInfo1@20 10002ed3 f   ThreadImpl.obj
 0001:00001eee       _Java_sun_management_ThreadImpl_getThreadTotalCpuTime0@16 10002eee f   ThreadImpl.obj
 0001:00001f07       _Java_sun_management_ThreadImpl_getThreadTotalCpuTime1@16 10002f07 f   ThreadImpl.obj
 0001:00001f20       _Java_sun_management_ThreadImpl_getThreadUserCpuTime0@16 10002f20 f   ThreadImpl.obj
 0001:00001f39       _Java_sun_management_ThreadImpl_getThreadUserCpuTime1@16 10002f39 f   ThreadImpl.obj
 0001:00001f52       _Java_sun_management_ThreadImpl_getThreads@8 10002f52 f   ThreadImpl.obj
 0001:00001f57       _Java_sun_management_ThreadImpl_getTotalThreadAllocatedMemory@8 10002f57 f   ThreadImpl.obj
 0001:00001f65       _Java_sun_management_ThreadImpl_resetContentionTimes0@16 10002f65 f   ThreadImpl.obj
 0001:00001f81       _Java_sun_management_ThreadImpl_resetPeakThreadCount0@8 10002f81 f   ThreadImpl.obj
 0001:00001f9f       _Java_sun_management_ThreadImpl_setThreadAllocatedMemoryEnabled0@12 10002f9f f   ThreadImpl.obj
 0001:00001fb4       _Java_sun_management_ThreadImpl_setThreadContentionMonitoringEnabled0@12 10002fb4 f   ThreadImpl.obj
 0001:00001fc9       _Java_sun_management_ThreadImpl_setThreadCpuTimeEnabled0@12 10002fc9 f   ThreadImpl.obj
 0001:00001fde       _Java_sun_management_VMManagementImpl_getAvailableProcessors@8 10002fde f   VMManagementImpl.obj
 0001:00001fe6       _Java_sun_management_VMManagementImpl_getClassInitializationTime@8 10002fe6 f   VMManagementImpl.obj
 0001:00001ff9       _Java_sun_management_VMManagementImpl_getClassLoadingTime@8 10002ff9 f   VMManagementImpl.obj
 0001:0000200c       _Java_sun_management_VMManagementImpl_getClassVerificationTime@8 1000300c f   VMManagementImpl.obj
 0001:0000201f       _Java_sun_management_VMManagementImpl_getDaemonThreadCount@8 1000301f f   VMManagementImpl.obj
 0001:00002032       _Java_sun_management_VMManagementImpl_getInitializedClassCount@8 10003032 f   VMManagementImpl.obj
 0001:00002045       _Java_sun_management_VMManagementImpl_getLiveThreadCount@8 10003045 f   VMManagementImpl.obj
 0001:00002058       _Java_sun_management_VMManagementImpl_getLoadedClassSize@8 10003058 f   VMManagementImpl.obj
 0001:0000206b       _Java_sun_management_VMManagementImpl_getMethodDataSize@8 1000306b f   VMManagementImpl.obj
 0001:0000207e       _Java_sun_management_VMManagementImpl_getPeakThreadCount@8 1000307e f   VMManagementImpl.obj
 0001:00002091       _Java_sun_management_VMManagementImpl_getProcessId@8 10003091 f   VMManagementImpl.obj
 0001:000020a7       _Java_sun_management_VMManagementImpl_getSafepointCount@8 100030a7 f   VMManagementImpl.obj
 0001:000020ba       _Java_sun_management_VMManagementImpl_getSafepointSyncTime@8 100030ba f   VMManagementImpl.obj
 0001:000020cd       _Java_sun_management_VMManagementImpl_getStartupTime@8 100030cd f   VMManagementImpl.obj
 0001:000020e0       _Java_sun_management_VMManagementImpl_getTotalApplicationNonStoppedTime@8 100030e0 f   VMManagementImpl.obj
 0001:000020f3       _Java_sun_management_VMManagementImpl_getTotalClassCount@8 100030f3 f   VMManagementImpl.obj
 0001:00002106       _Java_sun_management_VMManagementImpl_getTotalCompileTime@8 10003106 f   VMManagementImpl.obj
 0001:00002119       _Java_sun_management_VMManagementImpl_getTotalSafepointTime@8 10003119 f   VMManagementImpl.obj
 0001:0000212c       _Java_sun_management_VMManagementImpl_getTotalThreadCount@8 1000312c f   VMManagementImpl.obj
 0001:0000213f       _Java_sun_management_VMManagementImpl_getUnloadedClassCount@8 1000313f f   VMManagementImpl.obj
 0001:00002152       _Java_sun_management_VMManagementImpl_getUnloadedClassSize@8 10003152 f   VMManagementImpl.obj
 0001:00002165       _Java_sun_management_VMManagementImpl_getUptime0@8 10003165 f   VMManagementImpl.obj
 0001:00002178       _Java_sun_management_VMManagementImpl_getVerboseClass@8 10003178 f   VMManagementImpl.obj
 0001:00002189       _Java_sun_management_VMManagementImpl_getVerboseGC@8 10003189 f   VMManagementImpl.obj
 0001:0000219a       _Java_sun_management_VMManagementImpl_getVersion0@8 1000319a f   VMManagementImpl.obj
 0001:000021f0       _Java_sun_management_VMManagementImpl_getVmArguments0@8 100031f0 f   VMManagementImpl.obj
 0001:000021ff       _Java_sun_management_VMManagementImpl_initOptionalSupportFields@8 100031ff f   VMManagementImpl.obj
 0001:00002348       _Java_sun_management_VMManagementImpl_isThreadAllocatedMemoryEnabled@8 10003348 f   VMManagementImpl.obj
 0001:00002359       _Java_sun_management_VMManagementImpl_isThreadContentionMonitoringEnabled@8 10003359 f   VMManagementImpl.obj
 0001:0000236a       _Java_sun_management_VMManagementImpl_isThreadCpuTimeEnabled@8 1000336a f   VMManagementImpl.obj
 0001:000023ad       _sprintf                   100033ad f i VMManagementImpl.obj
 0001:000023c7       _JNI_OnLoad@8              100033c7 f   management.obj
 0001:00002425       _JVM_GetAllThreads@8       10003425 f   jvm:jvm.dll
 0001:0000242b       _JVM_ActiveProcessorCount@0 1000342b f   jvm:jvm.dll
 0001:00002431       _JVM_GetManagement@4       10003431 f   jvm:jvm.dll
 0001:00002437       _JNU_ThrowByName@12        10003437 f   java:java.dll
 0001:0000243d       _JNU_ThrowNullPointerException@8 1000343d f   java:java.dll
 0001:00002443       _JNU_ThrowOutOfMemoryError@8 10003443 f   java:java.dll
 0001:00002449       _JNU_NewObjectByName       10003449 f   java:java.dll
 0001:0000244f       _JNU_ThrowInternalError@8  1000344f f   java:java.dll
 0001:00002455       _JNU_ThrowIOException@8    10003455 f   java:java.dll
 0001:0000245b       _JNU_ThrowIOExceptionWithLastError@8 1000345b f   java:java.dll
 0001:00002461       _JNU_GetStringPlatformChars@12 10003461 f   java:java.dll
 0001:00002467       _JNU_ReleaseStringPlatformChars@12 10003467 f   java:java.dll
 0001:0000246d       _JNU_ThrowIllegalArgumentException@8 1000346d f   java:java.dll
 0001:00002473       _JNU_GetStaticFieldByName@20 10003473 f   java:java.dll
 0001:00002479       @__security_check_cookie@4 10003479 f   MSVCRT:secchk.obj
 0001:00002490       __allmul                   10003490 f   MSVCRT:llmul.obj
 0001:00002804       __DllMainCRTStartup@12     10003804 f   MSVCRT:dll_dllmain.obj
 0001:00002827       ___raise_securityfailure   10003827 f   MSVCRT:gs_report.obj
 0001:0000284f       ___report_gsfailure        1000384f f   MSVCRT:gs_report.obj
 0001:00002996       ___security_init_cookie    10003996 f   MSVCRT:gs_support.obj
 0001:000029e1       _DllMain@12                100039e1 f   MSVCRT:dll_dllmain_stub.obj
 0001:00002a03       ?__scrt_initialize_type_info@@YAXXZ 10003a03 f   MSVCRT:tncleanup.obj
 0001:00002a0f       ?__scrt_uninitialize_type_info@@YAXXZ 10003a0f f   MSVCRT:tncleanup.obj
 0001:00002a1b       ___local_stdio_scanf_options 10003a1b f i MSVCRT:default_local_stdio_options.obj
 0001:00002a21       ___scrt_initialize_default_local_stdio_options 10003a21 f   MSVCRT:default_local_stdio_options.obj
 0001:00002a82       ___scrt_acquire_startup_lock 10003a82 f   MSVCRT:utility.obj
 0001:00002ab4       ___scrt_dllmain_after_initialize_c 10003ab4 f   MSVCRT:utility.obj
 0001:00002adf       ___scrt_dllmain_before_initialize_c 10003adf f   MSVCRT:utility.obj
 0001:00002aed       ___scrt_dllmain_crt_thread_attach 10003aed f   MSVCRT:utility.obj
 0001:00002b0c       ___scrt_dllmain_crt_thread_detach 10003b0c f   MSVCRT:utility.obj
 0001:00002b19       ___scrt_dllmain_exception_filter 10003b19 f   MSVCRT:utility.obj
 0001:00002b4d       ___scrt_dllmain_uninitialize_c 10003b4d f   MSVCRT:utility.obj
 0001:00002b70       ___scrt_dllmain_uninitialize_critical 10003b70 f   MSVCRT:utility.obj
 0001:00002b7d       ___scrt_initialize_crt     10003b7d f   MSVCRT:utility.obj
 0001:00002bb6       ___scrt_initialize_onexit_tables 10003bb6 f   MSVCRT:utility.obj
 0001:00002c3d       ___scrt_is_nonwritable_in_current_image 10003c3d f   MSVCRT:utility.obj
 0001:00002cd1       ___scrt_release_startup_lock 10003cd1 f   MSVCRT:utility.obj
 0001:00002cee       ___scrt_uninitialize_crt   10003cee f   MSVCRT:utility.obj
 0001:00002d16       ___scrt_get_dyn_tls_init_callback 10003d16 f   MSVCRT:dyn_tls_init.obj
 0001:00002d1c       ___scrt_fastfail           10003d1c f   MSVCRT:utility_desktop.obj
 0001:00002e37       __crt_debugger_hook        10003e37 f   MSVCRT:utility_desktop.obj
 0001:00002e3f       __RTC_Initialize           10003e3f f   MSVCRT:initsect.obj
 0001:00002e6b       __RTC_Terminate            10003e6b f   MSVCRT:initsect.obj
 0001:00002ea0       __SEH_prolog4              10003ea0 f   MSVCRT:sehprolg4.obj
 0001:00002ee5       __except_handler4          10003ee5 f   MSVCRT:chandler4gs.obj
 0001:00002f14       @_guard_check_icall_nop@4  10003f14 f i MSVCRT:guard_support.obj
 0001:00002f17       ___isa_available_init      10003f17 f   MSVCRT:cpu_disp.obj
 0001:000030eb       __get_startup_argv_mode    100040eb f   MSVCRT:argv_mode.obj
 0001:000030ef       ___scrt_is_ucrt_dll_in_use 100040ef f   MSVCRT:ucrt_detection.obj
 0001:000030fb       _K32GetProcessMemoryInfo@12 100040fb f   kernel32:KERNEL32.dll
 0001:00003101       _strchr                    10004101 f   vcruntime:VCRUNTIME140.dll
 0001:00003107       _memset                    10004107 f   vcruntime:VCRUNTIME140.dll
 0001:0000310d       _strrchr                   1000410d f   vcruntime:VCRUNTIME140.dll
 0001:00003113       ___std_type_info_destroy_list 10004113 f   vcruntime:VCRUNTIME140.dll
 0001:00003119       __except_handler4_common   10004119 f   vcruntime:VCRUNTIME140.dll
 0001:0000311f       _strlen                    1000411f f   ucrt:api-ms-win-crt-string-l1-1-0.dll
 0001:00003125       __initterm                 10004125 f   ucrt:api-ms-win-crt-runtime-l1-1-0.dll
 0001:0000312b       __initterm_e               1000412b f   ucrt:api-ms-win-crt-runtime-l1-1-0.dll
 0001:00003131       __seh_filter_dll           10004131 f   ucrt:api-ms-win-crt-runtime-l1-1-0.dll
 0001:00003137       __configure_narrow_argv    10004137 f   ucrt:api-ms-win-crt-runtime-l1-1-0.dll
 0001:0000313d       __initialize_narrow_environment 1000413d f   ucrt:api-ms-win-crt-runtime-l1-1-0.dll
 0001:00003143       __initialize_onexit_table  10004143 f   ucrt:api-ms-win-crt-runtime-l1-1-0.dll
 0001:00003149       __execute_onexit_table     10004149 f   ucrt:api-ms-win-crt-runtime-l1-1-0.dll
 0001:0000314f       __cexit                    1000414f f   ucrt:api-ms-win-crt-runtime-l1-1-0.dll
 0001:00003155       ___acrt_initialize         10004155 f   MSVCRT:ucrt_stubs.obj
 0001:00003155       ___acrt_thread_attach      10004155 f   MSVCRT:ucrt_stubs.obj
 0001:00003155       ___acrt_thread_detach      10004155 f   MSVCRT:ucrt_stubs.obj
 0001:00003155       ___acrt_uninitialize       10004155 f   MSVCRT:ucrt_stubs.obj
 0001:00003155       ___acrt_uninitialize_critical 10004155 f   MSVCRT:ucrt_stubs.obj
 0001:00003155       ___scrt_stub_for_acrt_initialize 10004155 f   MSVCRT:ucrt_stubs.obj
 0001:00003155       ___scrt_stub_for_acrt_thread_attach 10004155 f   MSVCRT:ucrt_stubs.obj
 0001:00003155       ___scrt_stub_for_acrt_thread_detach 10004155 f   MSVCRT:ucrt_stubs.obj
 0001:00003155       ___scrt_stub_for_acrt_uninitialize 10004155 f   MSVCRT:ucrt_stubs.obj
 0001:00003155       ___scrt_stub_for_acrt_uninitialize_critical 10004155 f   MSVCRT:ucrt_stubs.obj
 0001:00003155       ___vcrt_initialize         10004155 f   MSVCRT:ucrt_stubs.obj
 0001:00003155       ___vcrt_thread_attach      10004155 f   MSVCRT:ucrt_stubs.obj
 0001:00003155       ___vcrt_thread_detach      10004155 f   MSVCRT:ucrt_stubs.obj
 0001:00003155       ___vcrt_uninitialize       10004155 f   MSVCRT:ucrt_stubs.obj
 0001:00003155       ___vcrt_uninitialize_critical 10004155 f   MSVCRT:ucrt_stubs.obj
 0001:00003158       ___scrt_stub_for_is_c_termination_complete 10004158 f   MSVCRT:ucrt_stubs.obj
 0001:00003158       __is_c_termination_complete 10004158 f   MSVCRT:ucrt_stubs.obj
 0001:0000315b       __filter_x86_sse2_floating_point_exception 1000415b f   MSVCRT:x86_exception_filter.obj
 0001:0000315b       __filter_x86_sse2_floating_point_exception_default 1000415b f   MSVCRT:x86_exception_filter.obj
 0002:00000000       __imp__GetSecurityDescriptorOwner@12 10005000     advapi32:ADVAPI32.dll
 0002:00000004       __imp__GetSecurityDescriptorDacl@16 10005004     advapi32:ADVAPI32.dll
 0002:00000008       __imp__GetAclInformation@16 10005008     advapi32:ADVAPI32.dll
 0002:0000000c       __imp__GetAce@12           1000500c     advapi32:ADVAPI32.dll
 0002:00000010       __imp__EqualSid@8          10005010     advapi32:ADVAPI32.dll
 0002:00000014       __imp__GetFileSecurityA@20 10005014     advapi32:ADVAPI32.dll
 0002:00000018       \177ADVAPI32_NULL_THUNK_DATA 10005018     advapi32:ADVAPI32.dll
 0002:0000001c       __imp__LoadLibraryA@4      1000501c     kernel32:KERNEL32.dll
 0002:00000020       __imp__GetProcAddress@8    10005020     kernel32:KERNEL32.dll
 0002:00000024       __imp__GetModuleFileNameA@12 10005024     kernel32:KERNEL32.dll
 0002:00000028       __imp__FreeLibrary@4       10005028     kernel32:KERNEL32.dll
 0002:0000002c       __imp__K32GetProcessMemoryInfo@12 1000502c     kernel32:KERNEL32.dll
 0002:00000030       __imp__IsDebuggerPresent@0 10005030     kernel32:KERNEL32.dll
 0002:00000034       __imp__InitializeSListHead@4 10005034     kernel32:KERNEL32.dll
 0002:00000038       __imp__DisableThreadLibraryCalls@4 10005038     kernel32:KERNEL32.dll
 0002:0000003c       __imp__UnhandledExceptionFilter@4 1000503c     kernel32:KERNEL32.dll
 0002:00000040       __imp__SetUnhandledExceptionFilter@4 10005040     kernel32:KERNEL32.dll
 0002:00000044       __imp__TerminateProcess@8  10005044     kernel32:KERNEL32.dll
 0002:00000048       __imp__IsProcessorFeaturePresent@4 10005048     kernel32:KERNEL32.dll
 0002:0000004c       __imp__QueryPerformanceCounter@4 1000504c     kernel32:KERNEL32.dll
 0002:00000050       __imp__GetSystemTimeAsFileTime@4 10005050     kernel32:KERNEL32.dll
 0002:00000054       __imp__GetVolumeInformationA@32 10005054     kernel32:KERNEL32.dll
 0002:00000058       __imp__GetLastError@0      10005058     kernel32:KERNEL32.dll
 0002:0000005c       __imp__InitializeCriticalSection@4 1000505c     kernel32:KERNEL32.dll
 0002:00000060       __imp__EnterCriticalSection@4 10005060     kernel32:KERNEL32.dll
 0002:00000064       __imp__LeaveCriticalSection@4 10005064     kernel32:KERNEL32.dll
 0002:00000068       __imp__GetProcessTimes@20  10005068     kernel32:KERNEL32.dll
 0002:0000006c       __imp__GetCurrentProcess@0 1000506c     kernel32:KERNEL32.dll
 0002:00000070       __imp__GetCurrentThreadId@0 10005070     kernel32:KERNEL32.dll
 0002:00000074       __imp__GlobalMemoryStatusEx@4 10005074     kernel32:KERNEL32.dll
 0002:00000078       __imp__GetSystemInfo@4     10005078     kernel32:KERNEL32.dll
 0002:0000007c       __imp__GetCurrentProcessId@0 1000507c     kernel32:KERNEL32.dll
 0002:00000080       \177KERNEL32_NULL_THUNK_DATA 10005080     kernel32:KERNEL32.dll
 0002:00000084       __imp__memset              10005084     vcruntime:VCRUNTIME140.dll
 0002:00000088       __imp__strrchr             10005088     vcruntime:VCRUNTIME140.dll
 0002:0000008c       __imp____std_type_info_destroy_list 1000508c     vcruntime:VCRUNTIME140.dll
 0002:00000090       __imp__strchr              10005090     vcruntime:VCRUNTIME140.dll
 0002:00000094       __imp___except_handler4_common 10005094     vcruntime:VCRUNTIME140.dll
 0002:00000098       \177VCRUNTIME140_NULL_THUNK_DATA 10005098     vcruntime:VCRUNTIME140.dll
 0002:0000009c       __imp___itoa               1000509c     ucrt:api-ms-win-crt-convert-l1-1-0.dll
 0002:0000009c       __imp__itoa                1000509c     ucrt:api-ms-win-crt-convert-l1-1-0.dll
 0002:000000a0       \177api-ms-win-crt-convert-l1-1-0_NULL_THUNK_DATA 100050a0     ucrt:api-ms-win-crt-convert-l1-1-0.dll
 0002:000000a4       __imp__calloc              100050a4     ucrt:api-ms-win-crt-heap-l1-1-0.dll
 0002:000000a8       __imp__free                100050a8     ucrt:api-ms-win-crt-heap-l1-1-0.dll
 0002:000000ac       __imp__malloc              100050ac     ucrt:api-ms-win-crt-heap-l1-1-0.dll
 0002:000000b0       \177api-ms-win-crt-heap-l1-1-0_NULL_THUNK_DATA 100050b0     ucrt:api-ms-win-crt-heap-l1-1-0.dll
 0002:000000b4       __imp___execute_onexit_table 100050b4     ucrt:api-ms-win-crt-runtime-l1-1-0.dll
 0002:000000b8       __imp___initialize_narrow_environment 100050b8     ucrt:api-ms-win-crt-runtime-l1-1-0.dll
 0002:000000bc       __imp___configure_narrow_argv 100050bc     ucrt:api-ms-win-crt-runtime-l1-1-0.dll
 0002:000000c0       __imp___seh_filter_dll     100050c0     ucrt:api-ms-win-crt-runtime-l1-1-0.dll
 0002:000000c4       __imp___initterm_e         100050c4     ucrt:api-ms-win-crt-runtime-l1-1-0.dll
 0002:000000c8       __imp___initterm           100050c8     ucrt:api-ms-win-crt-runtime-l1-1-0.dll
 0002:000000cc       __imp___cexit              100050cc     ucrt:api-ms-win-crt-runtime-l1-1-0.dll
 0002:000000d0       __imp___initialize_onexit_table 100050d0     ucrt:api-ms-win-crt-runtime-l1-1-0.dll
 0002:000000d4       __imp___getpid             100050d4     ucrt:api-ms-win-crt-runtime-l1-1-0.dll
 0002:000000d8       \177api-ms-win-crt-runtime-l1-1-0_NULL_THUNK_DATA 100050d8     ucrt:api-ms-win-crt-runtime-l1-1-0.dll
 0002:000000dc       __imp____stdio_common_vsprintf 100050dc     ucrt:api-ms-win-crt-stdio-l1-1-0.dll
 0002:000000e0       \177api-ms-win-crt-stdio-l1-1-0_NULL_THUNK_DATA 100050e0     ucrt:api-ms-win-crt-stdio-l1-1-0.dll
 0002:000000e4       __imp__strncpy             100050e4     ucrt:api-ms-win-crt-string-l1-1-0.dll
 0002:000000e8       __imp___strdup             100050e8     ucrt:api-ms-win-crt-string-l1-1-0.dll
 0002:000000e8       __imp__strdup              100050e8     ucrt:api-ms-win-crt-string-l1-1-0.dll
 0002:000000ec       __imp__strlen              100050ec     ucrt:api-ms-win-crt-string-l1-1-0.dll
 0002:000000f0       \177api-ms-win-crt-string-l1-1-0_NULL_THUNK_DATA 100050f0     ucrt:api-ms-win-crt-string-l1-1-0.dll
 0002:000000f4       __imp__clock               100050f4     ucrt:api-ms-win-crt-time-l1-1-0.dll
 0002:000000f8       \177api-ms-win-crt-time-l1-1-0_NULL_THUNK_DATA 100050f8     ucrt:api-ms-win-crt-time-l1-1-0.dll
 0002:000000fc       __imp__JNU_ThrowOutOfMemoryError@8 100050fc     java:java.dll
 0002:00000100       __imp__JNU_GetStaticFieldByName@20 10005100     java:java.dll
 0002:00000104       __imp__JNU_ThrowInternalError@8 10005104     java:java.dll
 0002:00000108       __imp__JNU_ThrowNullPointerException@8 10005108     java:java.dll
 0002:0000010c       __imp__JNU_ThrowIOExceptionWithLastError@8 1000510c     java:java.dll
 0002:00000110       __imp__JNU_GetStringPlatformChars@12 10005110     java:java.dll
 0002:00000114       __imp__JNU_ReleaseStringPlatformChars@12 10005114     java:java.dll
 0002:00000118       __imp__JNU_ThrowIllegalArgumentException@8 10005118     java:java.dll
 0002:0000011c       __imp__JNU_ThrowByName@12  1000511c     java:java.dll
 0002:00000120       __imp__JNU_ThrowIOException@8 10005120     java:java.dll
 0002:00000124       __imp__JNU_NewObjectByName 10005124     java:java.dll
 0002:00000128       \177java_NULL_THUNK_DATA   10005128     java:java.dll
 0002:0000012c       __imp__JVM_GetManagement@4 1000512c     jvm:jvm.dll
 0002:00000130       __imp__JVM_GetAllThreads@8 10005130     jvm:jvm.dll
 0002:00000134       __imp__JVM_ActiveProcessorCount@0 10005134     jvm:jvm.dll
 0002:00000138       \177jvm_NULL_THUNK_DATA    10005138     jvm:jvm.dll
 0002:0000013c       ___guard_check_icall_fptr  1000513c     MSVCRT:guard_support.obj
 0002:00000140       ___castguard_check_failure_os_handled_fptr 10005140     MSVCRT:guard_support.obj
 0002:00000144       ___xc_a                    10005144     MSVCRT:initializers.obj
 0002:00000148       ___xc_z                    10005148     MSVCRT:initializers.obj
 0002:0000014c       ___xi_a                    1000514c     MSVCRT:initializers.obj
 0002:00000150       ___xi_z                    10005150     MSVCRT:initializers.obj
 0002:00000154       ___xp_a                    10005154     MSVCRT:initializers.obj
 0002:00000158       ___xp_z                    10005158     MSVCRT:initializers.obj
 0002:0000015c       ___xt_a                    1000515c     MSVCRT:initializers.obj
 0002:00000160       ___xt_z                    10005160     MSVCRT:initializers.obj
 0002:00000170       ??_C@_0FA@KDGODBFA@JMX?5interface?5to?5diagnostic?5fra@ 10005170     DiagnosticCommandImpl.obj
 0002:000001c0       ??_C@_0CI@LDDEGNGM@java?1lang?1UnsupportedOperationE@ 100051c0     DiagnosticCommandImpl.obj
 0002:000001e8       ??_C@_0CN@GGIDBAIK@sun?1management?1DiagnosticComman@ 100051e8     DiagnosticCommandImpl.obj
 0002:00000218       ??_C@_0FA@HCGGLJHE@?$CILjava?1lang?1String?$DLLjava?1lang?1S@ 10005218     DiagnosticCommandImpl.obj
 0002:00000268       ??_C@_0BB@PPEHBGID@java?1util?1Arrays@ 10005268     DiagnosticCommandImpl.obj
 0002:0000027c       ??_C@_0CG@HHOJOFBP@?$CI?$FLLjava?1lang?1Object?$DL?$CJLjava?1util@ 1000527c     DiagnosticCommandImpl.obj
 0002:000002a4       ??_C@_06ECNHPIF@asList@    100052a4     DiagnosticCommandImpl.obj
 0002:000002ac       ??_C@_0BF@IEOOPILA@Invalid?5String?5Array@ 100052ac     DiagnosticCommandImpl.obj
 0002:000002c4       ??_C@_0CF@GOFCODGJ@sun?1management?1DiagnosticComman@ 100052c4     DiagnosticCommandImpl.obj
 0002:000002f0       ??_C@_0IB@BKJILNLP@?$CILjava?1lang?1String?$DLLjava?1lang?1S@ 100052f0     DiagnosticCommandImpl.obj
 0002:00000374       ??_C@_0O@PNKFDMOJ@Malformed?5UNC@ 10005374     FileSystemImpl.obj
 0002:00000384       ??_C@_0CA@CGFDCJE@Absolute?5filename?5not?5specified@ 10005384     FileSystemImpl.obj
 0002:000003a4       ??_C@_0BM@JPGKFFDK@GetVolumeInformation?5failed@ 100053a4     FileSystemImpl.obj
 0002:000003c0       ??_C@_0BH@EKMPGKNN@GetFileSecurity?5failed@ 100053c0     FileSystemImpl.obj
 0002:000003d8       ??_C@_0CC@PLIGLKOL@GetSecurityDescriptorOwner?5fail@ 100053d8     FileSystemImpl.obj
 0002:000003fc       ??_C@_0CB@EKBMIJAO@GetSecurityDescriptorDacl?5faile@ 100053fc     FileSystemImpl.obj
 0002:00000420       ??_C@_0CM@JFCPAEMB@Security?5descriptor?5does?5not?5co@ 10005420     FileSystemImpl.obj
 0002:0000044c       ??_C@_0BJ@OEDGCHLN@GetAclInformation?5failed@ 1000544c     FileSystemImpl.obj
 0002:00000468       ??_C@_0O@HNKFIIOB@GetAce?5failed@ 10005468     FileSystemImpl.obj
 0002:00000478       ??_C@_0CF@MADHDJEK@Lcom?1sun?1management?1VMOption$Or@ 10005478     Flag.obj
 0002:000004a0       ??_C@_0CD@CEAHIHPC@com?1sun?1management?1VMOption$Ori@ 100054a0     Flag.obj
 0002:000004c4       ??_C@_07MGCPDNLD@DEFAULT@  100054c4     Flag.obj
 0002:000004cc       ??_C@_0M@BODHNBPF@VM_CREATION@ 100054cc     Flag.obj
 0002:000004d8       ??_C@_0L@HNPILAMG@MANAGEMENT@ 100054d8     Flag.obj
 0002:000004e4       ??_C@_0M@FDANMCLI@ENVIRON_VAR@ 100054e4     Flag.obj
 0002:000004f0       ??_C@_0M@CEBLKBIO@CONFIG_FILE@ 100054f0     Flag.obj
 0002:000004fc       ??_C@_09ILMJHCBE@ERGONOMIC@ 100054fc     Flag.obj
 0002:00000508       ??_C@_05NNNMIPMB@OTHER@    10005508     Flag.obj
 0002:00000510       ??_C@_0BE@DONNLBPM@sun?1management?1Flag@ 10005510     Flag.obj
 0002:00000528       ??_C@_0EO@OCMOFBBM@?$CILjava?1lang?1String?$DLLjava?1lang?1O@ 10005528     Flag.obj
 0002:00000578       ??_C@_04LHKBAEFM@?$CIZ?$CJV@ 10005578     Flag.obj
 0002:00000580       ??_C@_0BC@DDPBLLCP@java?1lang?1Boolean@ 10005580     Flag.obj
 0002:00000594       ??_C@_04OHLIFDMD@?$CIJ?$CJV@ 10005594     Flag.obj
 0002:0000059c       ??_C@_0P@MLLHBNNC@java?1lang?1Long@ 1000559c     Flag.obj
 0002:000005ac       ??_C@_04HGHCEPA@?$CID?$CJV@ 100055ac     Flag.obj
 0002:000005b4       ??_C@_0BB@JKEOLFJD@java?1lang?1Double@ 100055b4     Flag.obj
 0002:000005c8       ??_C@_0CJ@FEKHENIJ@Number?5of?5Flag?5objects?5created?5@ 100055c8     Flag.obj
 0002:000005f4       ??_C@_0BO@EOMDLAMD@Invalid?5GarbageCollectorMBean@ 100055f4     GarbageCollectorImpl.obj
 0002:00000614       ??_C@_0P@CCHCOPNE@java?1lang?1Byte@ 10005614     GcInfoBuilder.obj
 0002:00000624       ??_C@_04CCAMHLCM@?$CIB?$CJV@ 10005624     GcInfoBuilder.obj
 0002:0000062c       ??_C@_0BC@OHJKABOO@java?1lang?1Integer@ 1000562c     GcInfoBuilder.obj
 0002:00000640       ??_C@_04PFANPMCN@?$CII?$CJV@ 10005640     GcInfoBuilder.obj
 0002:00000648       ??_C@_0BA@MBLENCLH@java?1lang?1Short@ 10005648     GcInfoBuilder.obj
 0002:00000658       ??_C@_04MKKJELNG@?$CIS?$CJV@ 10005658     GcInfoBuilder.obj
 0002:00000660       ??_C@_0BA@HJEPPKHG@java?1lang?1Float@ 10005660     GcInfoBuilder.obj
 0002:00000670       ??_C@_0BE@GKIHCGPM@java?1lang?1Character@ 10005670     GcInfoBuilder.obj
 0002:00000684       ??_C@_04JKLABMEJ@?$CIC?$CJV@ 10005684     GcInfoBuilder.obj
 0002:0000068c       ??_C@_0BH@KCPAAINP@Invalid?5num_attributes@ 1000568c     GcInfoBuilder.obj
 0002:000006a4       ??_C@_0BK@KGMIKEPP@Unexpected?5num_attributes@ 100056a4     GcInfoBuilder.obj
 0002:000006c0       ??_C@_0BG@HCNJLLGG@Invalid?5ext_att_count@ 100056c0     GcInfoBuilder.obj
 0002:000006d8       ??_C@_0BL@CHBGEDL@Unsupported?5attribute?5type@ 100056d8     GcInfoBuilder.obj
 0002:000006f8       ??_C@_0HO@LPKEKFAJ@?$CILsun?1management?1GcInfoBuilder?$DL@ 100056f8     GcInfoBuilder.obj
 0002:00000778       ??_C@_0BK@LAMMNKDJ@com?1sun?1management?1GcInfo@ 10005778     GcInfoBuilder.obj
 0002:00000794       ??_C@_0BJ@KKOPABNE@Memory?5Manager?5not?5found@ 10005794     MemoryManagerImpl.obj
 0002:000007b0       ??_C@_0BG@EJKNNBCK@Memory?5Pool?5not?5found@ 100057b0     MemoryPoolImpl.obj
 0002:000007f4       ??_C@_06NELKLDPM@?2?$CFs?2?$CFs@ 100057f4     OperatingSystemImpl.obj
 0002:000007fc       ??_C@_0L@MLLIHFJC@?2?$CFs?$CI?$CFs?$CJ?2?$CFs@ 100057fc     OperatingSystemImpl.obj
 0002:00000808       ??_C@_0O@JCGOHBMM@?2?$CFs?$CI?$CFs?$CD?$CFs?$CJ?2?$CFs@ 10005808     OperatingSystemImpl.obj
 0002:00000818       ??_C@_0P@CIDEDEDD@PdhAddCounterA@ 10005818     OperatingSystemImpl.obj
 0002:00000828       ??_C@_0O@HFNMDKII@PdhOpenQueryA@ 10005828     OperatingSystemImpl.obj
 0002:00000838       ??_C@_0O@EGDBAKJC@PdhCloseQuery@ 10005838     OperatingSystemImpl.obj
 0002:00000848       ??_C@_0BE@GPNBOCHE@PdhCollectQueryData@ 10005848     OperatingSystemImpl.obj
 0002:0000085c       ??_C@_0BM@EOJADGC@PdhGetFormattedCounterValue@ 1000585c     OperatingSystemImpl.obj
 0002:00000878       ??_C@_0BE@BJADGCJL@PdhEnumObjectItemsA@ 10005878     OperatingSystemImpl.obj
 0002:0000088c       ??_C@_0BB@EBECGLNG@PdhRemoveCounter@ 1000588c     OperatingSystemImpl.obj
 0002:000008a0       ??_C@_0BK@BKCEHIDJ@PdhLookupPerfNameByIndexA@ 100058a0     OperatingSystemImpl.obj
 0002:000008bc       ??_C@_02DPKJAMEF@?$CFd@    100058bc     OperatingSystemImpl.obj
 0002:000008c0       ??_C@_07OPODLDBJ@pdh?4dll@ 100058c0     OperatingSystemImpl.obj
 0002:000008c8       __real@3ff0000000000000    100058c8     OperatingSystemImpl.obj
 0002:000008d0       __real@4059000000000000    100058d0     OperatingSystemImpl.obj
 0002:000008d8       __real@bff0000000000000    100058d8     OperatingSystemImpl.obj
 0002:000008e0       __xmm@41f00000000000000000000000000000 100058e0     OperatingSystemImpl.obj
 0002:000008f0       ??_C@_05KBEOJPB@?$CFd?4?$CFd@ 100058f0     VMManagementImpl.obj
 0002:000008f8       ??_C@_01POHCFINO@Z@        100058f8     VMManagementImpl.obj
 0002:000008fc       ??_C@_0BK@DJAAMHIC@compTimeMonitoringSupport@ 100058fc     VMManagementImpl.obj
 0002:00000918       ??_C@_0CC@GDPMBOEP@threadContentionMonitoringSuppo@ 10005918     VMManagementImpl.obj
 0002:0000093c       ??_C@_0BM@GCPPCNJD@currentThreadCpuTimeSupport@ 1000593c     VMManagementImpl.obj
 0002:00000958       ??_C@_0BK@DMCEOMBH@otherThreadCpuTimeSupport@ 10005958     VMManagementImpl.obj
 0002:00000974       ??_C@_0BF@CHEGPANE@bootClassPathSupport@ 10005974     VMManagementImpl.obj
 0002:0000098c       ??_C@_0BK@EJFDBCBP@objectMonitorUsageSupport@ 1000598c     VMManagementImpl.obj
 0002:000009a8       ??_C@_0BJ@NIOHCHFH@synchronizerUsageSupport@ 100059a8     VMManagementImpl.obj
 0002:000009c4       ??_C@_0BN@GDBJIKMK@threadAllocatedMemorySupport@ 100059c4     VMManagementImpl.obj
 0002:000009e4       ??_C@_0CA@BBEOFMLC@remoteDiagnosticCommandsSupport@ 100059e4     VMManagementImpl.obj
 0002:00000a04       ??_C@_0BG@JBNOFFIK@gcNotificationSupport@ 10005a04     VMManagementImpl.obj
 0002:00000a1c       ??_C@_0BP@KJIDAONK@Unsupported?5Management?5version@ 10005a1c     management.obj
 0002:00000a3c       __pDefaultRawDllMain       10005a3c     MSVCRT:dll_dllmain.obj
 0002:00000a3c       __pRawDllMain              10005a3c     MSVCRT:dll_dllmain.obj
 0002:00000a48       __load_config_used         10005a48     MSVCRT:loadcfg.obj
 0002:00000b80       ___safe_se_handler_table   10005b80     <linker-defined>
 0002:00000b84       ___volatile_metadata       10005b84     <linker-defined>
 0002:00000ee4       ___rtc_iaa                 10005ee4     MSVCRT:initsect.obj
 0002:00000ee8       ___rtc_izz                 10005ee8     MSVCRT:initsect.obj
 0002:00000eec       ___rtc_taa                 10005eec     MSVCRT:initsect.obj
 0002:00000ef0       ___rtc_tzz                 10005ef0     MSVCRT:initsect.obj
 0002:00002938       __IMPORT_DESCRIPTOR_jvm    10007938     jvm:jvm.dll
 0002:0000294c       __IMPORT_DESCRIPTOR_java   1000794c     java:java.dll
 0002:00002960       __IMPORT_DESCRIPTOR_ADVAPI32 10007960     advapi32:ADVAPI32.dll
 0002:00002974       __IMPORT_DESCRIPTOR_KERNEL32 10007974     kernel32:KERNEL32.dll
 0002:00002988       __IMPORT_DESCRIPTOR_VCRUNTIME140 10007988     vcruntime:VCRUNTIME140.dll
 0002:0000299c       __IMPORT_DESCRIPTOR_api-ms-win-crt-heap-l1-1-0 1000799c     ucrt:api-ms-win-crt-heap-l1-1-0.dll
 0002:000029b0       __IMPORT_DESCRIPTOR_api-ms-win-crt-stdio-l1-1-0 100079b0     ucrt:api-ms-win-crt-stdio-l1-1-0.dll
 0002:000029c4       __IMPORT_DESCRIPTOR_api-ms-win-crt-string-l1-1-0 100079c4     ucrt:api-ms-win-crt-string-l1-1-0.dll
 0002:000029d8       __IMPORT_DESCRIPTOR_api-ms-win-crt-time-l1-1-0 100079d8     ucrt:api-ms-win-crt-time-l1-1-0.dll
 0002:000029ec       __IMPORT_DESCRIPTOR_api-ms-win-crt-runtime-l1-1-0 100079ec     ucrt:api-ms-win-crt-runtime-l1-1-0.dll
 0002:00002a00       __IMPORT_DESCRIPTOR_api-ms-win-crt-convert-l1-1-0 10007a00     ucrt:api-ms-win-crt-convert-l1-1-0.dll
 0002:00002a14       __NULL_IMPORT_DESCRIPTOR   10007a14     jvm:jvm.dll
 0003:00000040       ___security_cookie_complement 10009040     MSVCRT:gs_cookie.obj
 0003:00000044       ___security_cookie         10009044     MSVCRT:gs_cookie.obj
 0003:00000048       __fltused                  10009048     MSVCRT:fltused.obj
 0003:00000050       ___scrt_native_dllmain_reason 10009050     MSVCRT:utility.obj
 0003:00000060       ___isa_enabled             10009060     MSVCRT:cpu_disp.obj
 0003:00000064       ___scrt_ucrt_dll_is_in_use 10009064     MSVCRT:ucrt_stubs.obj
 0003:000000f8       _jmm_interface             100090f8     management.obj
 0003:000000fc       _jmm_version               100090fc     management.obj
 0003:00000100       _jvm                       10009100     management.obj
 0003:00000428       ?__type_info_root_node@@3U__type_info_node@@A 10009428     MSVCRT:tncleanup.obj
 0003:00000430       ?_OptionsStorage@?1??__local_stdio_scanf_options@@9@4_KA 10009430     MSVCRT:default_local_stdio_options.obj
 0003:00000438       ___scrt_current_native_startup_state 10009438     MSVCRT:utility.obj
 0003:0000043c       ___scrt_native_startup_lock 1000943c     MSVCRT:utility.obj
 0003:0000045c       ___scrt_debugger_hook_flag 1000945c     MSVCRT:utility_desktop.obj
 0003:00000460       ___isa_available           10009460     MSVCRT:cpu_disp.obj
 0003:00000464       ___favor                   10009464     MSVCRT:cpu_disp.obj
 0003:00000468       ?_OptionsStorage@?1??__local_stdio_printf_options@@9@9 10009468     <common>
 0003:00000470       ___dyn_tls_init_callback   10009470     <common>

 entry point at        0001:00002804

 Static symbols

 0000:ffff4000       .debug$S                   10000000     management.exp
 0000:ffff4000       .debug$S                   10000000     vcruntime:VCRUNTIME140.dll
 0000:ffff4000       .debug$S                   10000000     vcruntime:VCRUNTIME140.dll
 0000:ffff4000       .debug$S                   10000000     vcruntime:VCRUNTIME140.dll
 0000:ffff4000       .debug$S                   10000000     vcruntime:VCRUNTIME140.dll
 0000:ffff4000       .debug$S                   10000000     vcruntime:VCRUNTIME140.dll
 0000:ffff4000       .debug$S                   10000000     vcruntime:VCRUNTIME140.dll
 0000:ffff4000       .debug$S                   10000000     vcruntime:VCRUNTIME140.dll
 0000:ffff4000       .debug$S                   10000000     ucrt:api-ms-win-crt-convert-l1-1-0.dll
 0000:ffff4000       .debug$S                   10000000     ucrt:api-ms-win-crt-heap-l1-1-0.dll
 0000:ffff4000       .debug$S                   10000000     ucrt:api-ms-win-crt-heap-l1-1-0.dll
 0000:ffff4000       .debug$S                   10000000     ucrt:api-ms-win-crt-heap-l1-1-0.dll
 0000:ffff4000       .debug$S                   10000000     ucrt:api-ms-win-crt-runtime-l1-1-0.dll
 0000:ffff4000       .debug$S                   10000000     ucrt:api-ms-win-crt-runtime-l1-1-0.dll
 0000:ffff4000       .debug$S                   10000000     ucrt:api-ms-win-crt-runtime-l1-1-0.dll
 0000:ffff4000       .debug$S                   10000000     ucrt:api-ms-win-crt-runtime-l1-1-0.dll
 0000:ffff4000       .debug$S                   10000000     ucrt:api-ms-win-crt-runtime-l1-1-0.dll
 0000:ffff4000       .debug$S                   10000000     ucrt:api-ms-win-crt-runtime-l1-1-0.dll
 0000:ffff4000       .debug$S                   10000000     ucrt:api-ms-win-crt-runtime-l1-1-0.dll
 0000:ffff4000       .debug$S                   10000000     ucrt:api-ms-win-crt-runtime-l1-1-0.dll
 0000:ffff4000       .debug$S                   10000000     ucrt:api-ms-win-crt-runtime-l1-1-0.dll
 0000:ffff4000       .debug$S                   10000000     ucrt:api-ms-win-crt-runtime-l1-1-0.dll
 0000:ffff4000       .debug$S                   10000000     ucrt:api-ms-win-crt-runtime-l1-1-0.dll
 0000:ffff4000       .debug$S                   10000000     ucrt:api-ms-win-crt-runtime-l1-1-0.dll
 0000:ffff4000       .debug$S                   10000000     ucrt:api-ms-win-crt-runtime-l1-1-0.dll
 0000:ffff4000       .debug$S                   10000000     ucrt:api-ms-win-crt-runtime-l1-1-0.dll
 0000:ffff4000       .debug$S                   10000000     ucrt:api-ms-win-crt-stdio-l1-1-0.dll
 0000:ffff4000       .debug$S                   10000000     ucrt:api-ms-win-crt-string-l1-1-0.dll
 0000:ffff4000       .debug$S                   10000000     ucrt:api-ms-win-crt-string-l1-1-0.dll
 0000:ffff4000       .debug$S                   10000000     ucrt:api-ms-win-crt-string-l1-1-0.dll
 0000:ffff4000       .debug$S                   10000000     ucrt:api-ms-win-crt-time-l1-1-0.dll
 0000:ffff4000       .debug$S                   10000000     advapi32:ADVAPI32.dll
 0000:ffff4000       .debug$S                   10000000     advapi32:ADVAPI32.dll
 0000:ffff4000       .debug$S                   10000000     advapi32:ADVAPI32.dll
 0000:ffff4000       .debug$S                   10000000     advapi32:ADVAPI32.dll
 0000:ffff4000       .debug$S                   10000000     advapi32:ADVAPI32.dll
 0000:ffff4000       .debug$S                   10000000     advapi32:ADVAPI32.dll
 0000:ffff4000       .debug$S                   10000000     kernel32:KERNEL32.dll
 0000:ffff4000       .debug$S                   10000000     kernel32:KERNEL32.dll
 0000:ffff4000       .debug$S                   10000000     kernel32:KERNEL32.dll
 0000:ffff4000       .debug$S                   10000000     kernel32:KERNEL32.dll
 0000:ffff4000       .debug$S                   10000000     kernel32:KERNEL32.dll
 0000:ffff4000       .debug$S                   10000000     kernel32:KERNEL32.dll
 0000:ffff4000       .debug$S                   10000000     kernel32:KERNEL32.dll
 0000:ffff4000       .debug$S                   10000000     kernel32:KERNEL32.dll
 0000:ffff4000       .debug$S                   10000000     kernel32:KERNEL32.dll
 0000:ffff4000       .debug$S                   10000000     kernel32:KERNEL32.dll
 0000:ffff4000       .debug$S                   10000000     kernel32:KERNEL32.dll
 0000:ffff4000       .debug$S                   10000000     kernel32:KERNEL32.dll
 0000:ffff4000       .debug$S                   10000000     kernel32:KERNEL32.dll
 0000:ffff4000       .debug$S                   10000000     kernel32:KERNEL32.dll
 0000:ffff4000       .debug$S                   10000000     kernel32:KERNEL32.dll
 0000:ffff4000       .debug$S                   10000000     kernel32:KERNEL32.dll
 0000:ffff4000       .debug$S                   10000000     kernel32:KERNEL32.dll
 0000:ffff4000       .debug$S                   10000000     kernel32:KERNEL32.dll
 0000:ffff4000       .debug$S                   10000000     kernel32:KERNEL32.dll
 0000:ffff4000       .debug$S                   10000000     kernel32:KERNEL32.dll
 0000:ffff4000       .debug$S                   10000000     kernel32:KERNEL32.dll
 0000:ffff4000       .debug$S                   10000000     kernel32:KERNEL32.dll
 0000:ffff4000       .debug$S                   10000000     kernel32:KERNEL32.dll
 0000:ffff4000       .debug$S                   10000000     kernel32:KERNEL32.dll
 0000:ffff4000       .debug$S                   10000000     kernel32:KERNEL32.dll
 0000:ffff4000       .debug$S                   10000000     kernel32:KERNEL32.dll
 0000:ffff4000       .debug$S                   10000000     kernel32:KERNEL32.dll
 0000:ffff4000       .debug$S                   10000000     jvm:jvm.dll
 0000:ffff4000       .debug$S                   10000000     jvm:jvm.dll
 0000:ffff4000       .debug$S                   10000000     jvm:jvm.dll
 0000:ffff4000       .debug$S                   10000000     java:java.dll
 0000:ffff4000       .debug$S                   10000000     java:java.dll
 0000:ffff4000       .debug$S                   10000000     java:java.dll
 0000:ffff4000       .debug$S                   10000000     java:java.dll
 0000:ffff4000       .debug$S                   10000000     java:java.dll
 0000:ffff4000       .debug$S                   10000000     java:java.dll
 0000:ffff4000       .debug$S                   10000000     java:java.dll
 0000:ffff4000       .debug$S                   10000000     java:java.dll
 0000:ffff4000       .debug$S                   10000000     java:java.dll
 0000:ffff4000       .debug$S                   10000000     java:java.dll
 0000:ffff4000       .debug$S                   10000000     java:java.dll
 0001:00000454       _getFileDACL               10001454 f   FileSystemImpl.obj
 0001:0000049e       _getFileSecurityDescriptor 1000149e f   FileSystemImpl.obj
 0001:00000525       _isAccessUserOnly          10001525 f   FileSystemImpl.obj
 0001:000005d7       _isSecuritySupported       100015d7 f   FileSystemImpl.obj
 0001:000009e6       _find_origin_constant      100019e6 f   Flag.obj
 0001:0000111c       _EnterPdhCriticalSection   1000211c f   OperatingSystemImpl.obj
 0001:000013f8       _addCounter                100023f8 f   OperatingSystemImpl.obj
 0001:00001411       _allocateAndInitializePdhConstants 10002411 f   OperatingSystemImpl.obj
 0001:000014f7       _allocateCPUCounters       100024f7 f   OperatingSystemImpl.obj
 0001:00001530       _bindPdhFunctionPointers   10002530 f   OperatingSystemImpl.obj
 0001:000015f5       _currentQueryIndexForProcess 100025f5 f   OperatingSystemImpl.obj
 0001:000016f0       _deallocateCPUCounters     100026f0 f   OperatingSystemImpl.obj
 0001:000017c1       _getPdhProcessImageName    100027c1 f   OperatingSystemImpl.obj
 0001:00001866       _getPerformanceData        10002866 f   OperatingSystemImpl.obj
 0001:000018c8       _initializeCPUCounters     100028c8 f   OperatingSystemImpl.obj
 0001:00001a15       _initializeMultipleCounterForCPUs 10002a15 f   OperatingSystemImpl.obj
 0001:00001bbb       _initializePdhCPUCounters  10002bbb f   OperatingSystemImpl.obj
 0001:00001c2a       _lookupNameByIndex         10002c2a f   OperatingSystemImpl.obj
 0001:00001c8c       _makeFullCounterPath       10002c8c f   OperatingSystemImpl.obj
 0001:00001d58       _openQuery                 10002d58 f   OperatingSystemImpl.obj
 0001:00001d6b       _pdhCleanup                10002d6b f   OperatingSystemImpl.obj
 0001:00001d9e       _pdhInit                   10002d9e f   OperatingSystemImpl.obj
 0001:00001e1b       _pdhInitErrorHandler       10002e1b f   OperatingSystemImpl.obj
 0001:0000237b       _setStaticBooleanField     1000337b f   VMManagementImpl.obj
 0001:00002490       $$000000                   10003490     MSVCRT:llmul.obj
 0001:000024a9       hard                       100034a9     MSVCRT:llmul.obj
 0001:000024c4       ?dllmain_crt_dispatch@@YGHQAUHINSTANCE__@@KQAX@Z 100034c4 f   MSVCRT:dll_dllmain.obj
 0001:00002517       ?dllmain_crt_process_attach@@YAHQAUHINSTANCE__@@QAX@Z 10003517 f   MSVCRT:dll_dllmain.obj
 0001:0000261e       ?dllmain_crt_process_detach@@YAH_N@Z 1000361e f   MSVCRT:dll_dllmain.obj
 0001:000026ce       ?dllmain_dispatch@@YAHQAUHINSTANCE__@@KQAX@Z 100036ce f   MSVCRT:dll_dllmain.obj
 0001:000027d9       ?dllmain_raw@@YGHQAUHINSTANCE__@@KQAX@Z 100037d9 f   MSVCRT:dll_dllmain.obj
 0001:00002949       ___get_entropy             10003949 f   MSVCRT:gs_support.obj
 0001:00002a3e       ?find_pe_section@@YAPAU_IMAGE_SECTION_HEADER@@QAEI@Z 10003a3e f   MSVCRT:utility.obj
 0001:00002ea0       $$000000                   10003ea0     MSVCRT:sehprolg4.obj
 0002:000007c8       _MIN_UPDATE_INTERVAL       100057c8     OperatingSystemImpl.obj
 0002:000007cc       _PDH_PROCESSOR_IDX         100057cc     OperatingSystemImpl.obj
 0002:000007d0       _PDH_PROCESSOR_TIME_IDX    100057d0     OperatingSystemImpl.obj
 0002:000007d4       _PDH_PROCESS_IDX           100057d4     OperatingSystemImpl.obj
 0002:000007d8       _PDH_ID_PROCESS_IDX        100057d8     OperatingSystemImpl.obj
 0002:000007dc       _OBJECT_COUNTER_FMT        100057dc     OperatingSystemImpl.obj
 0002:000007e0       _OBJECT_COUNTER_FMT_LEN    100057e0     OperatingSystemImpl.obj
 0002:000007e4       _OBJECT_WITH_INSTANCES_COUNTER_FMT 100057e4     OperatingSystemImpl.obj
 0002:000007e8       _OBJECT_WITH_INSTANCES_COUNTER_FMT_LEN 100057e8     OperatingSystemImpl.obj
 0002:000007ec       _PROCESS_OBJECT_INSTANCE_COUNTER_FMT 100057ec     OperatingSystemImpl.obj
 0002:000007f0       _PROCESS_OBJECT_INSTANCE_COUNTER_FMT_LEN 100057f0     OperatingSystemImpl.obj
 0002:00000a40       _GS_ExceptionPointers      10005a40     MSVCRT:gs_report.obj
 0002:00000ef8       __sehtable$?dllmain_crt_process_attach@@YAHQAUHINSTANCE__@@QAX@Z 10005ef8     MSVCRT:dll_dllmain.obj
 0002:00000f18       __sehtable$?dllmain_crt_process_detach@@YAH_N@Z 10005f18     MSVCRT:dll_dllmain.obj
 0002:00000f40       __sehtable$?dllmain_dispatch@@YAHQAUHINSTANCE__@@KQAX@Z 10005f40     MSVCRT:dll_dllmain.obj
 0002:00000f60       __sehtable$___scrt_is_nonwritable_in_current_image 10005f60     MSVCRT:utility.obj
 0002:00000f80       .edata                     10005f80     management.exp
 0002:00000fa8       rgpv                       10005fa8     management.exp
 0002:00001128       rgszName                   10006128     management.exp
 0002:000012a8       rgwOrd                     100062a8     management.exp
 0002:00001368       szName                     10006368     management.exp
 0002:00001377       $N00001                    10006377     management.exp
 0002:00001385       $N00002                    10006385     management.exp
 0002:000013be       $N00003                    100063be     management.exp
 0002:00001405       $N00004                    10006405     management.exp
 0002:0000144c       $N00005                    1000644c     management.exp
 0002:0000148f       $N00006                    1000648f     management.exp
 0002:000014d4       $N00007                    100064d4     management.exp
 0002:00001500       $N00008                    10006500     management.exp
 0002:00001539       $N00009                    10006539     management.exp
 0002:00001575       $N00010                    10006575     management.exp
 0002:000015a1       $N00011                    100065a1     management.exp
 0002:000015c7       $N00012                    100065c7     management.exp
 0002:000015f8       $N00013                    100065f8     management.exp
 0002:0000161f       $N00014                    1000661f     management.exp
 0002:0000164c       $N00015                    1000664c     management.exp
 0002:00001678       $N00016                    10006678     management.exp
 0002:000016a2       $N00017                    100066a2     management.exp
 0002:000016ce       $N00018                    100066ce     management.exp
 0002:0000170d       $N00019                    1000670d     management.exp
 0002:0000174b       $N00020                    1000674b     management.exp
 0002:0000178f       $N00021                    1000678f     management.exp
 0002:000017c9       $N00022                    100067c9     management.exp
 0002:000017fe       $N00023                    100067fe     management.exp
 0002:0000183a       $N00024                    1000683a     management.exp
 0002:0000186e       $N00025                    1000686e     management.exp
 0002:000018aa       $N00026                    100068aa     management.exp
 0002:000018e8       $N00027                    100068e8     management.exp
 0002:0000191d       $N00028                    1000691d     management.exp
 0002:0000194f       $N00029                    1000694f     management.exp
 0002:00001982       $N00030                    10006982     management.exp
 0002:000019b2       $N00031                    100069b2     management.exp
 0002:000019eb       $N00032                    100069eb     management.exp
 0002:00001a25       $N00033                    10006a25     management.exp
 0002:00001a5e       $N00034                    10006a5e     management.exp
 0002:00001a92       $N00035                    10006a92     management.exp
 0002:00001ac2       $N00036                    10006ac2     management.exp
 0002:00001af8       $N00037                    10006af8     management.exp
 0002:00001b37       $N00038                    10006b37     management.exp
 0002:00001b76       $N00039                    10006b76     management.exp
 0002:00001bb0       $N00040                    10006bb0     management.exp
 0002:00001bea       $N00041                    10006bea     management.exp
 0002:00001c34       $N00042                    10006c34     management.exp
 0002:00001c7a       $N00043                    10006c7a     management.exp
 0002:00001cbb       $N00044                    10006cbb     management.exp
 0002:00001cf9       $N00045                    10006cf9     management.exp
 0002:00001d37       $N00046                    10006d37     management.exp
 0002:00001d74       $N00047                    10006d74     management.exp
 0002:00001dbb       $N00048                    10006dbb     management.exp
 0002:00001dfd       $N00049                    10006dfd     management.exp
 0002:00001e34       $N00050                    10006e34     management.exp
 0002:00001e64       $N00051                    10006e64     management.exp
 0002:00001e9d       $N00052                    10006e9d     management.exp
 0002:00001edd       $N00053                    10006edd     management.exp
 0002:00001f1a       $N00054                    10006f1a     management.exp
 0002:00001f57       $N00055                    10006f57     management.exp
 0002:00001f89       $N00056                    10006f89     management.exp
 0002:00001fc3       $N00057                    10006fc3     management.exp
 0002:00001ffd       $N00058                    10006ffd     management.exp
 0002:00002036       $N00059                    10007036     management.exp
 0002:0000206f       $N00060                    1000706f     management.exp
 0002:0000209c       $N00061                    1000709c     management.exp
 0002:000020dc       $N00062                    100070dc     management.exp
 0002:00002115       $N00063                    10007115     management.exp
 0002:0000214d       $N00064                    1000714d     management.exp
 0002:00002191       $N00065                    10007191     management.exp
 0002:000021da       $N00066                    100071da     management.exp
 0002:00002216       $N00067                    10007216     management.exp
 0002:00002255       $N00068                    10007255     management.exp
 0002:00002298       $N00069                    10007298     management.exp
 0002:000022d4       $N00070                    100072d4     management.exp
 0002:00002315       $N00071                    10007315     management.exp
 0002:00002352       $N00072                    10007352     management.exp
 0002:00002393       $N00073                    10007393     management.exp
 0002:000023ce       $N00074                    100073ce     management.exp
 0002:00002409       $N00075                    10007409     management.exp
 0002:00002443       $N00076                    10007443     management.exp
 0002:0000247e       $N00077                    1000747e     management.exp
 0002:000024b3       $N00078                    100074b3     management.exp
 0002:000024ed       $N00079                    100074ed     management.exp
 0002:0000252a       $N00080                    1000752a     management.exp
 0002:00002561       $N00081                    10007561     management.exp
 0002:000025ab       $N00082                    100075ab     management.exp
 0002:000025e6       $N00083                    100075e6     management.exp
 0002:00002622       $N00084                    10007622     management.exp
 0002:00002660       $N00085                    10007660     management.exp
 0002:0000269c       $N00086                    1000769c     management.exp
 0002:000026da       $N00087                    100076da     management.exp
 0002:00002717       $N00088                    10007717     management.exp
 0002:0000274a       $N00089                    1000774a     management.exp
 0002:00002782       $N00090                    10007782     management.exp
 0002:000027b7       $N00091                    100077b7     management.exp
 0002:000027eb       $N00092                    100077eb     management.exp
 0002:00002823       $N00093                    10007823     management.exp
 0002:00002865       $N00094                    10007865     management.exp
 0002:000028ac       $N00095                    100078ac     management.exp
 0002:000028f8       $N00096                    100078f8     management.exp
 0002:00002bb2       .idata$6                   10007bb2     jvm:jvm.dll
 0002:00002d18       .idata$6                   10007d18     java:java.dll
 0002:00002d9a       .idata$6                   10007d9a     advapi32:ADVAPI32.dll
 0002:00002fda       .idata$6                   10007fda     kernel32:KERNEL32.dll
 0002:00003040       .idata$6                   10008040     vcruntime:VCRUNTIME140.dll
 0002:00003166       .idata$6                   10008166     ucrt:api-ms-win-crt-heap-l1-1-0.dll
 0002:00003186       .idata$6                   10008186     ucrt:api-ms-win-crt-stdio-l1-1-0.dll
 0002:000031a6       .idata$6                   100081a6     ucrt:api-ms-win-crt-string-l1-1-0.dll
 0002:000031c8       .idata$6                   100081c8     ucrt:api-ms-win-crt-time-l1-1-0.dll
 0002:000031e8       .idata$6                   100081e8     ucrt:api-ms-win-crt-runtime-l1-1-0.dll
 0002:0000320a       .idata$6                   1000820a     ucrt:api-ms-win-crt-convert-l1-1-0.dll
 0003:00000000       ?class_name@?1??setLongValueAtObjectArray@@9@9 10009000     GcInfoBuilder.obj
 0003:00000004       ?signature@?1??setLongValueAtObjectArray@@9@9 10009004     GcInfoBuilder.obj
 0003:00000008       ?class_name@?1??setBooleanValueAtObjectArray@@9@9 10009008     GcInfoBuilder.obj
 0003:0000000c       ?signature@?1??setBooleanValueAtObjectArray@@9@9 1000900c     GcInfoBuilder.obj
 0003:00000010       ?class_name@?1??setByteValueAtObjectArray@@9@9 10009010     GcInfoBuilder.obj
 0003:00000014       ?signature@?1??setByteValueAtObjectArray@@9@9 10009014     GcInfoBuilder.obj
 0003:00000018       ?class_name@?1??setIntValueAtObjectArray@@9@9 10009018     GcInfoBuilder.obj
 0003:0000001c       ?signature@?1??setIntValueAtObjectArray@@9@9 1000901c     GcInfoBuilder.obj
 0003:00000020       ?class_name@?1??setShortValueAtObjectArray@@9@9 10009020     GcInfoBuilder.obj
 0003:00000024       ?signature@?1??setShortValueAtObjectArray@@9@9 10009024     GcInfoBuilder.obj
 0003:00000028       ?class_name@?1??setDoubleValueAtObjectArray@@9@9 10009028     GcInfoBuilder.obj
 0003:0000002c       ?signature@?1??setDoubleValueAtObjectArray@@9@9 1000902c     GcInfoBuilder.obj
 0003:00000030       ?class_name@?1??setFloatValueAtObjectArray@@9@9 10009030     GcInfoBuilder.obj
 0003:00000034       ?signature@?1??setFloatValueAtObjectArray@@9@9 10009034     GcInfoBuilder.obj
 0003:00000038       ?class_name@?1??setCharValueAtObjectArray@@9@9 10009038     GcInfoBuilder.obj
 0003:0000003c       ?signature@?1??setCharValueAtObjectArray@@9@9 1000903c     GcInfoBuilder.obj
 0003:00000068       _default_origin            10009068     Flag.obj
 0003:0000006c       _vm_creation_origin        1000906c     Flag.obj
 0003:00000070       _mgmt_origin               10009070     Flag.obj
 0003:00000074       _envvar_origin             10009074     Flag.obj
 0003:00000078       _config_file_origin        10009078     Flag.obj
 0003:0000007c       _ergo_origin               1000907c     Flag.obj
 0003:00000080       _other_origin              10009080     Flag.obj
 0003:00000088       _main_process              10009088     OperatingSystemImpl.obj
 0003:0000008c       _PdhAddCounter_i           1000908c     OperatingSystemImpl.obj
 0003:00000090       _PdhOpenQuery_i            10009090     OperatingSystemImpl.obj
 0003:00000094       _PdhCloseQuery_i           10009094     OperatingSystemImpl.obj
 0003:00000098       _PdhCollectQueryData_i     10009098     OperatingSystemImpl.obj
 0003:0000009c       _PdhGetFormattedCounterValue_i 1000909c     OperatingSystemImpl.obj
 0003:000000a0       _PdhEnumObjectItems_i      100090a0     OperatingSystemImpl.obj
 0003:000000a4       _PdhRemoveCounter_i        100090a4     OperatingSystemImpl.obj
 0003:000000a8       _PdhLookupPerfNameByIndex_i 100090a8     OperatingSystemImpl.obj
 0003:000000ac       _initializationLock        100090ac     OperatingSystemImpl.obj
 0003:000000cc       _pdhProcessImageName       100090cc     OperatingSystemImpl.obj
 0003:000000d0       _pdhIDProcessCounterFmt    100090d0     OperatingSystemImpl.obj
 0003:000000d4       _numberOfJavaProcessesAtInitialization 100090d4     OperatingSystemImpl.obj
 0003:000000d8       _processTotalCPULoad       100090d8     OperatingSystemImpl.obj
 0003:000000dc       _multiCounterCPULoad       100090dc     OperatingSystemImpl.obj
 0003:000000e0       _cpuFactor                 100090e0     OperatingSystemImpl.obj
 0003:000000e8       _numCpus                   100090e8     OperatingSystemImpl.obj
 0003:000000ec       ?myPid@?1??getProcessID@@9@9 100090ec     OperatingSystemImpl.obj
 0003:000000f0       ?initialized@?1??pdhInit@@9@9 100090f0     OperatingSystemImpl.obj
 0003:000000f4       ?initialized@?1??initializePdhCPUCounters@@9@9 100090f4     OperatingSystemImpl.obj
 0003:00000104       ?__proc_attached@@3HA      10009104     MSVCRT:dll_dllmain.obj
 0003:00000108       _GS_ExceptionRecord        10009108     MSVCRT:gs_report.obj
 0003:00000158       _GS_ContextRecord          10009158     MSVCRT:gs_report.obj
 0003:00000440       ?is_initialized_as_dll@@3_NA 10009440     MSVCRT:utility.obj
 0003:00000441       ?module_local_atexit_table_initialized@@3_NA 10009441     MSVCRT:utility.obj
 0003:00000444       ?module_local_atexit_table@@3U_onexit_table_t@@A 10009444     MSVCRT:utility.obj
 0003:00000450       ?module_local_at_quick_exit_table@@3U_onexit_table_t@@A 10009450     MSVCRT:utility.obj
 0004:00000060       $R000000                   1000a060     management.dll.res
